:1000000012C017C52AC029C028C07FC426C025C079
:100010006BC4CAC322C0DDC220C0AAC21EC01DC09C
:1000200089C521C51AC011241FBECFE5D4E0DEBFAB
:10003000CDBF10E0A0E6B0E0E4E1F1E102C0059040
:100040000D92A637B107D9F713E0A6E7B0E001C0DB
:100050001D92A23AB107E1F708C1D2CF20918500E5
:1000600080916100821710F4282FAB9A8091830051
:10007000909184008338910560F01BBC1ABC19BCB8
:1000800018BC13BCAB9A01979093840080938300B3
:100090000895822F9927880F991F9BBD8ABD99BD0E
:1000A00088BD23BD089582E08FBD81E485BD85B301
:1000B000817F85BB89E08EBD089592B7980F82B786
:1000C000891B87FDFCCF0895AF92BF92CF92DF923C
:1000D000EF92FF920F931F93CF93DF93182F8CE231
:1000E000A82E81E0B82EC12CD12C439885E090E059
:1000F0009093860080938500B1DF09D688EC90E06C
:10010000A3D3C12FDD27D0938600C0938500EE24B2
:10011000FF248701EA14FB040C051D0578F4809187
:100120006D00882311F42ED201C024D384E6C5DFEC
:100130000894E11CF11C011D111DECCFC601B50195
:100140002FE030E040E050E0C3D7A21AB30AC40A5F
:10015000D50A0894A108B108C108D10889E1A816F8
:10016000B104C104D104C8F0D2D5809198008F5F4A
:10017000809398008091980066E08AD790939800C9
:1001800074D3D0938600C093850068DF449BBFCFB3
:1001900082B390E8892782BBBACFDF91CF911F91BC
:1001A0000F91FF90EF90DF90CF90BF90AF900895A8
:1001B00060E070E080917F00882379F580918E0067
:1001C000882349F1209190003091910041E02D3237
:1001D000340708F09B01293C310510F028EC30E091
:1001E0002B303105F0F08CEF90E0289FA001299F83
:1001F000500D389F500D1124CA01885D994064EB61
:1002000070E052D76D5F7F4F6F3F710551F048F03E
:100210006FEF70E006C0AB9A05C080919003682F25
:100220007727AB98862F9927089580918300909126
:1002300084009093770380937603809182009927BE
:100240009093790380937803809176009091770062
:1002500090937B0380937A0380919000909191001A
:1002600090937D0380937C030895CAE3D4E0DEBFBE
:10027000CDBFDE011196E8E6F0E085E001900D9239
:100280008150E1F7782E88E084BB85BB8AEB81BB87
:1002900080E882BB8EE087BB81E088BB57D2BAD2B0
:1002A000789480E180936E0000E010E00130110549
:1002B00009F4979A86E990E0C7D297988AEF90E080
:1002C000C3D20F5F1F4F0530110584F305E010E026
:1002D00084EF91E0B9D23AD2E6DE80916E0080934D
:1002E0008803809185008093890310928A038AEAAB
:1002F00080938B0310928C0380E5AAD3E8D285E625
:1003000090E08ED286E690E08BD287E690E088D2AD
:100310007C018EEF90E084D24C018DEE93E080D290
:100320006C018EEE93E07CD25C01C70182D28823FF
:10033000E1F3979A10928600109285008FDE88E094
:1003400080BF81E087B98AE090E06AD27C0181E0D9
:1003500090E090937903809378031092910010922B
:100360009000809185008093890380919800871583
:1003700051F0109262001092630082E390E050D23C
:100380007C01709098008091850090918600892B67
:1003900061F410927A0010926300C6014AD2882359
:1003A00071F081E0809362000AC08091620088232E
:1003B00019F081E080937A008CED95E031D24EDE29
:1003C000809163008F5F80936300813051F680914C
:1003D0006200882311F0979A01C0979826DF8091D8
:1003E0006D00882311F4CED001C0C4D1C40121D244
:1003F000882339F182E390E013D24C01809182008E
:10040000482F5527209183003091840042175307CD
:1004100010F48F5F04C02417350718F481508093BF
:1004200082008091820090916100823428F0915086
:1004300090936100AB9A05C09F3F19F09F5F909326
:100440006100C601F6D1882319F18AE090E0E8D175
:100450006C012091780030917900C901880F991FB3
:10046000880F991F820F931F820F931F66E070E021
:100470001BD67093770060937600109279001092EB
:10048000780080918E00882319F481E080936000C9
:10049000C501CFD1882391F18CED95E0C1D15C01EC
:1004A00002301105B9F0033011053CF401151105B6
:1004B00059F00130110559F01FC00330110569F0E2
:1004C0000430110599F018C082E390E008C082E87A
:1004D00090E005C08CE390E002C08CE890E090933F
:1004E0008600809385000F5F1F4F08C086E990E06B
:1004F000909386008093850000E010E0C70199D1B9
:10050000882331F08091760090917700892B29F033
:1005100080917A00882309F424CF81E080936200DF
:10052000439884E690E07CD17C0180917A00882316
:1005300009F417CFAB9810927A008AE0C5DD1092CB
:1005400062008091980081508093980088B18A6001
:1005500088B984E690E064D17C01C7016AD1882320
:10056000E1F384E690E05CD17C0197E0792EF9CE4E
:100570001F920F920FB60F9211240F900FBE0F9083
:100580001F9018955E9B24C080916D008823E1F434
:100590008091890090918A00019690938A008093BF
:1005A0008900FC01E656FD4FE081ED3019F08436FC
:1005B000910539F410928A001092890081E08093AD
:1005C0006D00589AECB9089510928A001092890033
:1005D00008951F920F920FB60F9211248F938CB132
:1005E000809388008F910F900FBE0F901F901895E9
:1005F000AC01A0E0B0E09D01A817B90748F4EAE912
:10060000F2E08191280F311D1196A417B507C8F3A8
:100610003F70FD01E656FD4FC90146E0969587956E
:100620004A95E1F7835C80831196FD01E656FD4F04
:100630002F733070822F835C8083A556BD4F8DE071
:100640008C9310926D0080919A028CB908951F933B
:10065000CF93DF93382FEA01722F10E083E280936B
:100660009A0260939B0230939C02A3E0B0E0772350
:1006700009F458C0772311F4972F07C0FE01E10F4A
:10068000F11D1F5F9081715011F4472F0EC0FE01C4
:10069000E10FF11D1F5F4081715039F0FE01E10F44
:1006A000F11D1F5F6081715001C0672FFD01E6568B
:1006B000FD4F892F86958695835C80831196FD0179
:1006C000E656FD4F892F99278370907024E0880F9C
:1006D000991F2A95E1F755279A0194E036952795B9
:1006E0009A95E1F7822B835C80831196FD01E65693
:1006F000FD4F4F705070440F551F440F551F862FEC
:10070000992756E0969587955A95E1F7842B835C57
:1007100080831196FD01E656FD4F6F73635C608325
:100720001196A5CFCD0164DFDF91CF911F91089580
:10073000CF93C82F8A3011F48DE0FADF5D9BFECF96
:10074000CCB980E090E0CF910895089588E18AB90E
:10075000599A80E189B960E070E088E993E03BD381
:1007600088EC90E05DD09093FF028093FE028AE2D5
:100770008CB908958091FE029091FF025AD088238F
:1007800091F080916D00882371F022E244E653E0FD
:100790006091990284E45BDF82E390E041D0909322
:1007A000FF028093FE0208951F920F920FB60F92E0
:1007B00011248F939F93809186038F5F809386038C
:1007C00080918D00815080938D008F3FE1F483E014
:1007D00080938D0080918B0090918C000196909376
:1007E0008C0080938B0080917F00882319F08150CA
:1007F00080937F0080918E00882329F080918E0065
:10080000815080938E009F918F910F900FBE0F901B
:100810001F90189582E083BF89B7816089BF0895D2
:1008200020918B0030918C00280F391FC90101974E
:10083000089520918B0030918C00821B930B892F9F
:100840009927807899270895CF93DF93E9DFEC010A
:10085000CE01EFDF8823E1F3DF91CF91089586EA9F
:1008600086B987E087B9369A089527B196E097B997
:1008700010BE83ED86B9349A97B9369A349BFECF71
:1008800027B944B155B1440F551F440F551F493C7A
:10089000510510F048EC50E0809183009091840065
:1008A0009C0163E0220F331F6A95E1F7281B390B87
:1008B000420F531F83E0569547958A95E1F7509371
:1008C00084004093830016B888E080BF08958EB5F9
:1008D000806C8EBD8EB580648EBD89B7806289BF05
:1008E00089B7846089BF08951F920F920FB60F9247
:1008F00011248F9380918F008F5F80938F008F9151
:100900000F900FBE0F901F9018951F920F920FB669
:100910000F9211242F933F938F939F930EB406FE53
:100920000FC010928F0086B597B590939300809377
:1009300092008EB58F7B8EBD84E680938E0070C052
:100940008EB580648EBD26B537B5809192009091AA
:100950009300281B390B80918F009927982F8827A7
:10096000990F280F391F689414F836952795169417
:10097000E1F730939500209394002851314030F4F2
:1009800088E191E0909395008093940020919400E9
:100990003091950028513140309395002093940078
:1009A00080919000909191008217930730F480918C
:1009B00090009091910001960CC0809190009091D0
:1009C00091002817390748F4809190009091910088
:1009D0000197909391008093900020919000309126
:1009E0009100C901880F991F880F991F880F991FBF
:1009F000821B930B2091940030919500820F931FDE
:100A000023E0969587952A95E1F79093950080933A
:100A10009400909391008093900081E08093600017
:100A20009F918F913F912F910F900FBE0F901F902C
:100A300018951F920F920FB60F9211248F938AB7B9
:100A40008F7B8ABF8F910F900FBE0F901F901895CC
:100A500082B986B7856486BF86B78F7D86BF8FEFE4
:100A60008093870308951F920F920FB60F9211245F
:100A70002F938F939F93EF93FF9381B199278038A2
:100A80009105A1F08138910524F48036910541F05B
:100A900045C0883A910549F1883B910531F13EC046
:100AA00085EC86BF8FEF809387033AC023B1909186
:100AB00087039F3F49F4109287032093960080910B
:100AC0006E00281759F10FC0E92FFF27E057FC4FA0
:100AD00020839F5F9093870382E380937F0094300D
:100AE000E8F01092870385E81AC0909196008091F3
:100AF0006E00981789F490918703E92FFF27E85734
:100B0000FC4F808183B9892F8F5F80938703883062
:100B100028F01092870302C08FEF83B985EC86BF5F
:100B2000FF91EF919F918F912F910F900FBE0F909A
:100B30001F9018951F920F920FB60F9211242F93AA
:100B40003F934F935F936F937F938F939F93AF9355
:100B5000BF93EF93FF93979A8091980099278230E3
:100B6000910509F44AC0833091052CF4009779F07F
:100B7000019759F1B8C08430910509F476C08430EA
:100B800091050CF458C0059709F486C0ACC082EA00
:100B90008FBD81E685BD88E087BB459B11C082B3D0
:100BA000877E82BB959A8091600081115EDE81E034
:100BB00087B9809198008F5F80939800409883C098
:100BC00082B3877D82BB949A8EC082B3877E82BBBC
:100BD000959A45990CC082EA8FBD81E485BD8CE071
:100BE00087BB80916000811140DE17B836C082EA71
:100BF0008FBD81E685BD88E075C082EA8FBD81E446
:100C000085BD8CE087BB459B11C082B38F7C82BBC6
:100C1000939A80916000811128DE82E087B9409824
:100C2000809198008F5F809398004DC082B3877E3B
:100C300082BB959A58C082B38F7C82BB939A4599A8
:100C40000EC082EA8FBD81E485BD8AE087BB8091BA
:100C5000600081110ADE81E087B9409AE1CF82EA23
:100C60008FBD81E485BD8CE03DC082EA8FBD81E40B
:100C700085BD8AE087BB459B0AC082B3877D82BB66
:100C8000949A809160008111F0DD17B8C8CF82B3CB
:100C90008F7C82BB939A27C082B3877D82BB949A54
:100CA00045991BC082EA8FBD81E685BD88E087BB80
:100CB00081E084BD809160008111D7DD82E087B939
:100CC000409A109298008091780090917900019656
:100CD000909379008093780006C082EA8FBD81E40A
:100CE00085BD8AE087BB979810926000FF91EF91D5
:100CF000BF91AF919F918F917F916F915F914F9134
:100D00003F912F910F900FBE0F901F9018958091DB
:100D1000980099278230910551F1833091052CF488
:100D2000009769F00197B9F0089584309105D1F1E9
:100D3000843091054CF1059709F441C0089582EA89
:100D40008FBD81E685BD88E087BB82B3877D82BB8E
:100D5000949A82E032C082EA8FBD81E685BD88E048
:100D600087BB82B3877E82BB959A81E018C082EAF6
:100D70008FBD81E485BD8CE087BB82B3877E82BB5B
:100D8000959A17B8409A089582EA8FBD81E485BD8F
:100D90008CE087BB82B38F7C82BB939A82E087B959
:100DA0004098089582EA8FBD81E485BD8AE087BBC3
:100DB00082B38F7C82BB939A81E087B9E3CF82EACA
:100DC0008FBD81E485BD8AE087BB82B3877D82BB0E
:100DD000949A17B8E5CF0F931F93CF93DF938C01AD
:100DE000EB01009711F4672BB9F16EE070E081E040
:100DF00090E037D0FC01892B71F180E88383209744
:100E000071F0D387C28781E88383809198039091A2
:100E10009903892B21F4F0939903E093980301152A
:100E20001105C9F0118700878381826083838091D7
:100E30009A0390919B03892B71F4F0939B03E093A9
:100E40009A0380919C0390919D03892B21F4F09348
:100E50009D03E0939C03CF01DF91CF911F910F91F0
:100E600008950F931F93CF93DF93869F8001879FF1
:100E7000100D969F100D1124C8010DD0EC010097A4
:100E800021F0A80160E070E0FCD0CE01DF91CF91AD
:100E90001F910F910895CF93DF93AC01029710F447
:100EA00042E050E020E030E0A091A003B091A10327
:100EB000BD01F901109709F44CC08D919C911197D7
:100EC0008417950731F14817590738F42115310572
:100ED00019F08217930708F49C01FD01A281B381E8
:100EE000109759F721153105A1F1C901841B950B04
:100EF000049708F4A901DB01E0E0F0E0109749F164
:100F00008D919C91119782179307F9F4421753071B
:100F100079F4ED018A819B81309719F09383828364
:100F200004C09093A1038093A003CD0102964AC010
:100F3000241B350BFD01E20FF31F41935193225007
:100F400030402D933C93CF013DC0FD01A281B38180
:100F5000D5CF80919E0390919F03892B41F480917E
:100F600072009091730090939F0380939E03E09191
:100F70007000F0917100309741F4EDB7FEB78091A9
:100F8000740090917500E81BF90BA0919E03B0913D
:100F90009F039F012A1B3B0B2417350788F0CA01CA
:100FA00002962817390760F0CD01840F951F02962D
:100FB00090939F0380939E034D935D93CD0102C058
:100FC00080E090E0DF91CF910895CF93DF93009779
:100FD00009F454C0DC011297ED011B821A82809142
:100FE000A0039091A103009721F1FC0140E050E0A3
:100FF000EA17FB0718F1ED01FB83EA832D913C9181
:101000001197C20FD31FCE0102968E179F0771F45E
:101010008A819B81280F391F2E5F3F4F11963C9389
:101020002E9382819381FD01938382834115510523
:1010300059F4B093A103A093A00320C0AF01028094
:10104000F381E02D3097A1F6EA01BB83AA83CA01A0
:10105000029628813981820F931F8A179B0771F4AA
:101060008D919C911197280F391F2E5F3F4F398327
:101070002883FD01828193819B838A83DF91CF91B5
:101080000895DC0101C06D9341505040E0F7089590
:10109000991B79E004C0991F961708F0961B881FCA
:1010A0007A95C9F780950895AA1BBB1B51E107C02B
:1010B000AA1FBB1FA617B70710F0A61BB70B881FE8
:1010C000991F5A95A9F780959095BC01CD01089577
:1010D000A1E21A2EAA1BBB1BFD010DC0AA1FBB1F3C
:1010E000EE1FFF1FA217B307E407F50720F0A21BAE
:1010F000B30BE40BF50B661F771F881F991F1A941B
:1011000069F760957095809590959B01AC01BD0144
:04111000CF0108956E
:1011140001FF01010A00FF004D6F696E0001406488
:061124000000A203200000
:00000001FF
